:020000040000fa
:080000000002040000000000f2
:020000040000fa
:040008009a03000057
:020000040000fa
:04000c00b403000039
:020000040000fa
:040010006603000083
:020000040000fa
:04001400ce03000017
:020000040000fa
:04001800e8030000f9
:020000040000fa
:04001c0032030000ab
:020000040000fa
:040020008003000059
:020000040000fa
:040024004c03000089
:020000040000fa
:040028003c04000094
:020000040000fa
:04002c003c04000090
:020000040000fa
:040030003c0400008c
:020000040000fa
:040034003c04000088
:020000040000fa
:040038003c04000084
:020000040000fa
:04003c003c04000080
:020000040000fa
:040040003c0400007c
:020000040000fa
:040044003c04000078
:020000040000fa
:040048003c04000074
:020000040000fa
:04004c003c04000070
:020000040000fa
:040050003c0400006c
:020000040000fa
:040054003c04000068
:020000040000fa
:040058003c04000064
:020000040000fa
:04005c003c04000060
:020000040000fa
:040060003c0400005c
:020000040000fa
:040064003c04000058
:020000040000fa
:040068003c04000054
:020000040000fa
:04006c003c04000050
:020000040000fa
:040070003c0400004c
:020000040000fa
:040074003c04000048
:020000040000fa
:040078003c04000044
:020000040000fa
:04007c003c04000040
:020000040000fa
:040080003c0400003c
:020000040000fa
:040084003c04000038
:020000040000fa
:040088003c04000034
:020000040000fa
:04008c003c04000030
:020000040000fa
:040090003c0400002c
:020000040000fa
:040094003c04000028
:020000040000fa
:040098003c04000024
:020000040000fa
:04009c003c04000020
:020000040000fa
:0400a0003c0400001c
:020000040000fa
:0400a4003c04000018
:020000040000fa
:0400a8003c04000014
:020000040000fa
:0400ac003c04000010
:020000040000fa
:0400b0003c0400000c
:020000040000fa
:0400b4003c04000008
:020000040000fa
:0400b8003c04000004
:020000040000fa
:0400bc003c04000000
:020000040000fa
:0400c0003c040000fc
:020000040000fa
:0400c4003c040000f8
:020000040000fa
:0400c8003c040000f4
:020000040000fa
:0400cc003c040000f0
:020000040000fa
:0400d0003c040000ec
:020000040000fa
:0400d4003c040000e8
:020000040000fa
:0400d8003c040000e4
:020000040000fa
:0400dc003c040000e0
:020000040000fa
:0400e0003c040000dc
:020000040000fa
:0400e4003c040000d8
:020000040000fa
:0400e8003c040000d4
:020000040000fa
:0400ec003c040000d0
:020000040000fa
:0400f0003c040000cc
:020000040000fa
:0400f4003c040000c8
:020000040000fa
:0400f8003c040000c4
:020000040000fa
:0400fc003c040000c0
:020000040000fa
:040100003c040000bb
:020000040000fa
:040104003c040000b7
:020000040000fa
:040108003c040000b3
:020000040000fa
:04010c003c040000af
:020000040000fa
:040110003c040000ab
:020000040000fa
:040114003c040000a7
:020000040000fa
:040118003c040000a3
:020000040000fa
:04011c003c0400009f
:020000040000fa
:040120003c0400009b
:020000040000fa
:040124003c04000097
:020000040000fa
:040128003c04000093
:020000040000fa
:04012c003c0400008f
:020000040000fa
:040130003c0400008b
:020000040000fa
:040134003c04000087
:020000040000fa
:040138003c04000083
:020000040000fa
:04013c003c0400007f
:020000040000fa
:040140003c0400007b
:020000040000fa
:040144003c04000077
:020000040000fa
:040148003c04000073
:020000040000fa
:04014c003c0400006f
:020000040000fa
:040150003c0400006b
:020000040000fa
:040154003c04000067
:020000040000fa
:040158003c04000063
:020000040000fa
:04015c003c0400005f
:020000040000fa
:040160003c0400005b
:020000040000fa
:040164003c04000057
:020000040000fa
:040168003c04000053
:020000040000fa
:04016c003c0400004f
:020000040000fa
:040170003c0400004b
:020000040000fa
:040174003c04000047
:020000040000fa
:040178003c04000043
:020000040000fa
:04017c003c0400003f
:020000040000fa
:040180003c0400003b
:020000040000fa
:040184003c04000037
:020000040000fa
:040188003c04000033
:020000040000fa
:04018c003c0400002f
:020000040000fa
:040190003c0400002b
:020000040000fa
:040194003c04000027
:020000040000fa
:04019800020400005d
:020000040000fa
:04019c003c0400001f
:020000040000fa
:0401a0003c0400001b
:020000040000fa
:0401a4003c04000017
:020000040000fa
:0401a8003c04000013
:020000040000fa
:0401ac003c0400000f
:020000040000fa
:0401b0003c0400000b
:020000040000fa
:0401b4003c04000007
:020000040000fa
:0401b8003c04000003
:020000040000fa
:0401bc003c040000ff
:020000040000fa
:0401c0003c040000fb
:020000040000fa
:0401c4003c040000f7
:020000040000fa
:0401c8003c040000f3
:020000040000fa
:0401cc003c040000ef
:020000040000fa
:0401d0003c040000eb
:020000040000fa
:0401d4003c040000e7
:020000040000fa
:0401d8003c040000e3
:020000040000fa
:0401dc003c040000df
:020000040000fa
:0401e0003c040000db
:020000040000fa
:0401e4003c040000d7
:020000040000fa
:0401e8003c040000d3
:020000040000fa
:0401ec003c040000cf
:020000040000fa
:0401f0003c040000cb
:020000040000fa
:0401f4003c040000c7
:020000040000fa
:0401f8003c040000c3
:020000040000fa
:0401fc003c040000bf
:020000040000fa
:040200003c040000ba
:020000040000fa
:040204003c040000b6
:020000040000fa
:040208003c040000b2
:020000040000fa
:04020c003c040000ae
:020000040000fa
:040210003c040000aa
:020000040000fa
:040214003c040000a6
:020000040000fa
:040218003c040000a2
:020000040000fa
:04021c003c0400009e
:020000040000fa
:040220003c0400009a
:020000040000fa
:040224003c04000096
:020000040000fa
:040228003c04000092
:020000040000fa
:04022c003c0400008e
:020000040000fa
:040230003c0400008a
:020000040000fa
:040234003c04000086
:020000040000fa
:040238003c04000082
:020000040000fa
:04023c003c0400007e
:020000040000fa
:040240003c0400007a
:020000040000fa
:040244003c04000076
:020000040000fa
:040248003c04000072
:020000040000fa
:04024c003c0400006e
:020000040000fa
:040250003c0400006a
:020000040000fa
:040254003c04000066
:020000040000fa
:040258003c04000062
:020000040000fa
:04025c003c0400005e
:020000040000fa
:040260003c0400005a
:020000040000fa
:040264003c04000056
:020000040000fa
:040268003c04000052
:020000040000fa
:04026c003c0400004e
:020000040000fa
:040270003c0400004a
:020000040000fa
:040274003c04000046
:020000040000fa
:040278003c04000042
:020000040000fa
:04027c003c0400003e
:020000040000fa
:040280003c0400003a
:020000040000fa
:040284003c04000036
:020000040000fa
:040288003c04000032
:020000040000fa
:04028c003c0400002e
:020000040000fa
:040290003c0400002a
:020000040000fa
:040294003c04000026
:020000040000fa
:040298003c04000022
:020000040000fa
:04029c003c0400001e
:020000040000fa
:0402a0003c0400001a
:020000040000fa
:0402a4003c04000016
:020000040000fa
:0402a8003c04000012
:020000040000fa
:0402ac003c0400000e
:020000040000fa
:0402b0003c0400000a
:020000040000fa
:0402b4003c04000006
:020000040000fa
:0402b8003c04000002
:020000040000fa
:0402bc003c040000fe
:020000040000fa
:0402c0003c040000fa
:020000040000fa
:0402c4003c040000f6
:020000040000fa
:0402c8003c040000f2
:020000040000fa
:0402cc003c040000ee
:020000040000fa
:0402d0003c040000ea
:020000040000fa
:0402d4003c040000e6
:020000040000fa
:0402d8003c040000e2
:020000040000fa
:0402dc003c040000de
:020000040000fa
:0402e0003c040000da
:020000040000fa
:0402e4003c040000d6
:020000040000fa
:0402e8003c040000d2
:020000040000fa
:0402ec003c040000ce
:020000040000fa
:0402f0003c040000ca
:020000040000fa
:0402f4003c040000c6
:020000040000fa
:0402f8003c040000c2
:020000040000fa
:0402fc003c040000be
:020000040000fa
:040300003c040000b9
:020000040000fa
:040304003c040000b5
:020000040000fa
:040308003c040000b1
:020000040000fa
:04030c003c040000ad
:020000040000fa
:040310003c040000a9
:020000040000fa
:040314003c040000a5
:020000040000fa
:040318003c040000a1
:020000040000fa
:04031c003c0400009d
:020000040000fa
:040320003c04000099
:020000040000fa
:040324003c04000095
:020000040000fa
:040328003c04000091
:020000040000fa
:04032c003c0400008d
:020000040000fa
:100400006f0921000eff24000e018800000000008b
:10041000000020000000e000020032000001200087
:100420002002880014000700150107000000e0000a
:1004300003003a00203722000100200002003700ac
:100440000000200001002000810f70000100320038
:100450000f000700000020000000e0000200320052
:1004600000000200000000004a2902000000000015
:100470000040da000000fe00200020000000e00044
:1004800002003200100020009001880000000600e9
:10049000a1028800800478000000eb001f003700f4
:1004a000e284440054a0b4009905ba00e2844400f8
:1004b00054a0b4009906ba00e284440054a0b400e9
:1004c0000006eb00476fde00fd07b200ae018800ba
:1004d000636ce10003003a000ad801000000eb0061
:1004e0000e003700606ce10008003a00004deb00a0
:1004f0000a05e800020039003420ec000af0a000f0
:100500008b05e900f9ff3e00040037006168e10057
:10051000010032000086eb000b00070019c7ba008b
:100520001905ba000e04e00003003a000a00e000da
:10053000dbff3a0000000600fe07b200ae028800b2
:100540008a047800f5ff37000cd0a300e20f4d00bd
:100550001c00390089027800354dba000a05e80010
:10056000020039003420ec000af0a0008b05e900fd
:100570000f003200254dba000a05e80002003900dc
:100580003420ec000af0a0008b05e90008003200de
:100590000c00e0000600320015cdba000a05e800a4
:1005a000020039003420ec000af0a0008b05e900bd
:1005b0008984e80054a0b4000b00e000e2ff3a0098
:1005c000000006009902ba00055d78008b05e9007d
:1005d000f7ff3200c82ade00055d78008b05e900d0
:1005e000f3ff32000c00e000f1ff320019ddba0029
:1005f000eeff3700742e040000000000dc2e040023
:1006000000000000501904000000000090220400c7
:1006100000000000f8220400000000001023040085
:1006200000000000121c0400000000005c27040011
:1006300000000000d227040000000000ea270400a8
:1006400000000000641d0400000000000a280400ef
:10065000000000008028040000000000982804002a
:10066000000000003600f800809fbe00829fbe00a0
:10067000849fbe00869fbe0000082000c4150700ae
:100680004f03be004f02be004f01be004f00be0030
:100690003600f900004006003600f800809fbe00da
:1006a000829fbe00849fbe00869fbe00000820007f
:1006b000b71507004f03be004f02be004f01be003a
:1006c0004f00be003600f900004006003600f8007a
:1006d000809fbe00829fbe00849fbe00869fbe009a
:1006e00000042000aa1507004f03be004f02be0001
:1006f0004f01be004f00be003600f900004006006a
:100700003600f800809fbe00829fbe00849fbe001e
:10071000869fbe00000220009d1507004f03be000b
:100720004f02be004f01be004f00be003600f90070
:10073000004006003600f800809fbe00829fbe0089
:10074000849fbe00869fbe00100020009015070009
:100750004f03be004f02be004f01be004f00be005f
:100760003600f900004006003600f800809fbe0009
:10077000829fbe00849fbe00869fbe002000200096
:10078000831507004f03be004f02be004f01be009d
:100790004f00be003600f900004006003600f800a9
:1007a000809fbe00829fbe00849fbe00869fbe00c9
:1007b00040002000761507004f03be004f02be0028
:1007c0004f01be004f00be003600f9000040060099
:1007d0003600f800809fbe00829fbe00849fbe004e
:1007e000869fbe0080002000691507004f03be00f1
:1007f0004f02be004f01be004f00be003600f900a0
:10080000004006003600f8003200f8003400f8001e
:1008100010002000a00188001000200000d0fe0081
:100820003e8ea800e00125001010a0001189820072
:10083000e088820001000100b18982008089820085
:1008400001000100518a8200208a8200010001001b
:100850000000000000000000000000000000000098
:100860000b88a9003e8ea9003400f9003200f9007f
:100870003600f900004006000040da000000fe00eb
:04088000000005006f
:020000040000fa
:100884001000fa00889fbe000004780010002000c9
:10089400e0b79f000000eb00f0b79f006000b800d5
:1008a40080bf9f0091bf9f00a0bf9f00b1bf9f006a
:1008b400c0bf9f00d1bf9f001800e00002003d00b0
:1008c4001838a30014003a00980078006180600092
:1008d4000004e0000d003a000000eb001004980052
:1008e400180090008000eb00e90f5000e08f5800e2
:1008f400100036000000eb00100498006fb0970061
:100904004f04be000080fa00000006001000200022
:1009140010049800f2ff37001878a300f0ff3200ab
:1009240098007800618060000004e000f7ff3a005e
:10093400e9ff370000060100420137001f013700bc
:1009440005013700f2003700650037004400370026
:10095400360037001e003700010037004b01370016
:10096400f810900028b89000808f5000a502320043
:100974001880a000f810900028b89000808f5000d4
:10098400b1013900f810900028b89000808f500011
:10099400daff360028b89000c810900000804000ac
:1009a40020bc9800a8b8900078109000808f500068
:1009b400d2ff36007810900020bc98006fb09700ea
:1009c4004f04be000080fa0000000600cfff37008d
:1009d4001880a00078009000880890000001e800ca
:1009e40072049800810f5000c4ff3600800020007c
:1009f40010049800080890000000e80070049800b3
:100a040028e891000004e000bcff3200a00e2000a2
:100a140008004000391307006fb097004f04be0070
:100a24000080fa0000000600b8ff3700681090004c
:100a3400e20f5000bb01320078b89000e8b8900093
:100a440020c1900021c09800c808de0030c1900089
:100a540031c098007000200010049800a7ff3700f0
:100a64001880a00078b89000104090000078a3008f
:100a7400cd01320038109000c81090000080400072
:100a840030149800b810900028b89000808f50005f
:100a94009aff360028b890003014980078b8900077
:100aa400410f200088804000206190002160980060
:100ab400c808de0030619000316098006810900032
:100ac4000000e000e3ff320068109000e20f5000e5
:100ad4008aff3a00600020001004980087ff370066
:100ae4001880a0000000eb0030149800800f200054
:100af400600c980078b89000610220008880400063
:100b04002061900021609800c808de0030619000e8
:100b140031609800581890003014980068109000c4
:100b2400e20f5000b6013200d81890001828900047
:100b3400808f5000e9003200e818900038309000af
:100b4400808f5000e50032009830900068199000c2
:100b540038309000000051000100b80080bf9f00b1
:100b640091bf9f000fb897009fb89700283190005d
:100b7400700111000201e900030033008100d1007b
:100b84000080d300fbff370080bf9f0091bf9f0010
:100b9400f820900058199000182890000000510087
:100ba4000100b800a0bf9f00b1bf9f002fb89700fd
:100bb400bfb8970008299000700111000201e900f4
:100bc400030033008100d1000080d300fbff370015
:100bd400a0bf9f00b1bf9f00789190000fb897000d
:100be4009fb897000200b800c0bf9f00d1bf9f000c
:100bf4002fb99700bfb997004fba9700dfba970093
:100c04000500090042aad8008000eb00c0bf9f0085
:100c1400d1bf9f002fb99700bfb997000fb89700b5
:100c24009fb89700800f5100818f5900fb01360057
:100c3400789090004fb99700dfb997008000eb00df
:100c44000200500083805800c0bf9f00d1bf9f00a6
:100c5400b810900048119000200320008090b90043
:100c64000100400030149800681090000000e0007b
:100c7400a1003a0058b990004fb89700dfb8970028
:100c8400cf91de00800f5100818f5900d1013600d1
:100c940058b89000cf80de00c0bf9f00d1bf9f0036
:100ca400b80191004fba9700dfba970078b8900066
:100cb400040178008000eb000300010078b8900084
:100cc400a05090008180fb00305090004800dd006f
:100cd400008070004fb99700dfb9970002087800d0
:100ce40078b89000a05890008180fb0030589000a4
:100cf4004800dd00008070004fb99700dfb997000d
:100d0400020878005000200010049800fbfe370011
:100d14001880a00028009000b80090000001e800ae
:100d240022049800810f5000f4fe36003800900031
:100d34000000e80020049800400020001848a300a8
:100d4400edfe3a006fb097004f04be000080fa0039
:100d540000000600edfe37001880a1001800e00036
:100d640003003d0018e8a3000100320018d0a000e1
:100d740008e091000004e00018013a001800e000c7
:100d8400defe3d0018d8a300dcfe32001818a300d4
:100d9400dafe32001828a300d8fe32001878a30027
:100da400d6fe3a001848a300d4fe320018d0a100a1
:100db4003000200010049800d0fe37001880a000f6
:100dc40008007800e9100700efb097000100600008
:100dd400e0b79f00f8b89000114090000074a100a3
:100de400904098009800910078b8900001000100ac
:100df40078b89000205190000281fb00b050900020
:100e0400c808dd008100710078b8900000c190002e
:100e14000281fb0010c090004800dd0082087000d1
:100e240050828200e20f5000ff00320028e8910057
:100e34000004e00093003a00200020001004980011
:100e4400aefe37001880a0000000eb0020049800dc
:100e5400700498001830a1001810a1001898a3007d
:100e6400770032001840a10028e891000004e00057
:100e740003003200a00e2000080040004d120700bd
:100e840010002000100498009cfe37000800780031
:100e94004f0f0700efb0970001006000e0b79f001c
:100ea400f8b89000114090000074a10090409800a0
:100eb40068109000e20f5000770032003800900074
:100ec4000000e80020049800080890000000e800f2
:100ed4007004980010002000eaff37002898900062
:100ee4008000eb00c0bf9f00d1bf9f00681090003e
:100ef4000000e0005fff320068109000e20f500035
:100f040080ff3a000000eb00f0b79f00808282006f
:100f1400ffb09700808f50007aff31007fb09700b8
:100f2400f400b90000004400700191004fb897002c
:100f3400dfb89700cf91de00800f5100818f5900f8
:100f4400120136007fb09700f400b900000044009d
:100f540070009100cf80de00c0bf9f00d1bf9f0012
:100f64007fb09700f400b90000004400d00991005c
:100f74004fba9700dfba97007fb09700f400b9002a
:100f84000000440010089100040178008000eb0088
:100f9400030001007fb09700f400b9000000440092
:100fa40010089100a05090008180fb003050900008
:100fb4004800dd00008070004fb99700dfb997004a
:100fc400020878007fb09700f400b90000004400e4
:100fd40010089100a05890008180fb0030589000c8
:100fe4004800dd00008070000c0032007fb09700e4
:100ff400f400b9000000440010089100a0589000cb
:101004008180fb00305890004800dd0000807000b3
:101014004fb99700dfb99700020878007fb09700b6
:101024000000e800f0b79f00818282007fb0970043
:10103400808f5000b9ff3e005000200032ff37007f
:101044001840a00088ff3700a8b89000481090000e
:101054000080500020bc9800a8b890007810900040
:10106400808f500025fe3100f810900021bc9800bc
:101074006fb097004f04be000080fa000000060025
:1010840022fe3700a00e200008004000c91107000e
:101094002000200069ff37000000eb00f0b79f003c
:1010a40018189000ffb09700808f500083ff310024
:1010b4007fb09700f400b90000004400900891004c
:1010c400114090000074a100904098007fb09700f8
:1010d4000000e800f0b79f00981890007fb09700d8
:1010e400808f500075ff36007fb09700f400b90080
:1010f4000000440090089100114090000074a10089
:10110400904098007fb097000000e800f0b79f007f
:10111400981890007fb09700808f5000e4ff3e0045
:1011240066ff37001880a00078b89000a0c0900037
:101134008180fb0030c190004811dd000281700005
:10114400f80890008100410020c1900021c098005f
:10115400c808de0030c1900031c0980078b8900013
:1011640020c190000281fb00b0c09000c808dd00df
:1011740081007100a0492000808f5000dffd3600ff
:101184000000e80060bc980078b89000e8b89000cf
:1011940020c1900021c09800c808de0030c1900032
:1011a40031c098002bfe3700080078007b10070040
:1011b400efb0970001006000e0b79f006810900056
:1011c4000000e000a0003a00f8b890001140900040
:1011d4000074a0009040980026fe3700dd890a00c4
:1011e40018000000000e200008004000191207003b
:1011f40080c46400dd090a0018000000dffe370027
:10120400e808900061bc980078b89000e8b89000b5
:1012140020c1900021c09800c808de0030c19000b1
:1012240031c0980040fe37000000eb00f0b79f008b
:1012340080828200ffb09700808f5000fbfe310057
:101244007fb09700f400b9000000440090089100ba
:10125400114090000074a100904098007fb0970066
:10126400f400b90000004400b00891007fb097007a
:10127400f400b900000044001008910001000100ce
:101284007fb09700f400b9000000440010089100fa
:10129400205190000281fb00b0509000c808dd008e
:1012a400810071007fb09700f400b9000000440091
:1012b4001008910000c190000281fb0010c0900052
:1012c4004800dd00820870007fb097000000e8004d
:1012d400f0b79f00818282007fb09700808f50001a
:1012e400d2fe36007fb09700f400b900000044003d
:1012f40090089100114090000074a1009040980063
:101304007fb09700f400b90000004400b0089100d9
:101314007fb09700f400b900000044001008910069
:10132400010001007fb09700f400b9000000440000
:1013340010089100205190000281fb00b0509000f1
:10134400c808dd00810071007fb09700f400b90087
:10135400000044001008910000c190000281fb00cd
:1013640010c090004800dd00820870007fb0970034
:101374000000e800f0b79f00818282007fb09700f0
:10138400808f5000aeff3e00a8fe37007fb097006c
:10139400f400b90000004400000991004fb8970020
:1013a400dfb897008001eb00800f5100818f590056
:1013b400ebfe31007fb09700f400b9000000440058
:1013c400000891008000eb00c0bf9f00d1bf9f00c8
:1013d400e3fe370068b990004fb89700dfb8970074
:1013e4008001eb00800f5100818f59002cfe3100e9
:1013f40068b890008000eb00c0bf9f00d1bf9f0081
:1014040027fe37001880a1006fb097004f04be007c
:101414000080fa00000006003cfd37002898900088
:101424008000eb00c0bf9f00d1bf9f00b8109000a8
:1014340048119000200320008090b9000100400072
:101444003014980008fe370068109000e20f500036
:1014540088fd3a00f8b89000114090000074a00094
:10146400904098000000eb00f0b79f00981890009f
:101474007fb09700808f50007efd36007fb09700cc
:10148400f400b9000000440090089100114090005d
:101494000074a000904098007fb097000000e8001e
:0414a400f1ff37001d
:020000040000fa
:1014a800f6874700889fbe008a9fbe008c9fbe00bb
:1014b8008e1f780010002000f0af9f004a11250011
:1014c8000004eb00080d780060bd200090888a00b9
:1014d800e400450050b62f008008780066074500f4
:1014e800b0492000000f7800b8888a00e804450059
:1014f800c01b2500800c78006a0145000395210077
:10150800030978000329220013898a00832f220007
:1015180003898a000331220023898a001201780096
:10152800f1b79f00020001001900780002c22000f4
:10153800a0419000224098004811de00b041900080
:1015480032409800190078001a017800fa0f20003c
:1015580080499000024898004811de0090499000a8
:1015680012489800190078004041900042c0b3002a
:1015780042409800d04190005840980019007800e7
:10158800e041900000c6eb006c409800f0419000ec
:10159800fbc7b3007b40980019007800a049900071
:1015a80028489800b04990003848980019007800f9
:1015b8008051900008509800905190001850980061
:1015c80019007800c049900042489800504990009e
:1015d8005848980019007800604990006c489800b5
:1015e800704990007b489800190078006a8144008f
:1015f8008a026100a0519000255098004812de0030
:10160800b05190003450980019007800805990002b
:1016180008589800905990001858980019007800b8
:10162800c051900048509800d051900058509800f0
:1016380019007800e05190006c509800f05190002b
:101648007b50980019007800fe8644008a81660065
:10165800a3b79f00a0599000cfe3970027589800a0
:10166800c869de0093b79f00b0599000afe39700b8
:101678003758980019007800806190000860980039
:10168800906190001860980019007800c059900087
:1016980048589800d0599000585898001900780078
:1016a800e05990006c589800f05990007b589800c9
:1016b8001900780003f32f00898141000a83610033
:1016c800a063900026609800c819de00306390007f
:1016d8003360980019007800ffb0970091007800f7
:1016e80080c1900001c09800c808de0090c1900039
:1016f80011c09800190078009e007800a0c19000e1
:1017080021c09800c808de00b0c1900031c0980020
:1017180019007800c0c0900048c09800d0c0900060
:1017280058c0980019007800e0c0900068c0980080
:10173800f0c0900078c098001900780080c8900028
:1017480008c8980090c8900018c898001900780038
:10175800a0c8900028c89800b0c8900038c8980061
:1017680019007800c0c8900048c89800d0c89000f8
:1017780058c8980019007800e0c8900068c8980018
:10178800f0c8900078c8980019007800c1f32f00bd
:10179800898040008a81600000d3900003d09800bf
:1017a800c808de0090d1900011d098001900780088
:1017b800c0d0900048d09800d0d0900058d0980061
:1017c80019007800e0d0900068d09800f0d0900020
:1017d80078d098001900780080d8900008d8980030
:1017e80090d8900018d8980019007800a0d89000d8
:1017f80028d89800b0d8900038d8980019007800f8
:10180800c0e0900048e09800d0e0900058e09800d0
:1018180019007800e0e0900068e09800f0e090009f
:1018280078e098001900780080e8900008e89800af
:1018380090e8900018e8980019007800a0e8900057
:1018480028e89800b0e8900038e8980099007800f7
:10185800114090000074a100904098009900780011
:10186800114090000054a100904098009900780021
:10187800114090000044a100904098009900780021
:10188800114090000064a100904098001900780071
:101898001004a100190078001014a1009900780024
:1018a800114090000034a100904098006e07470056
:1018b80000802000000f7800810f200001097800c7
:1018c800f0814400071420008709780072814400e1
:1018d8000090210000097800e400510000c82000b1
:1018e80080087800f484440080222500800c780069
:1018f8006403410027c12100070b7800c775220047
:10190800b7898a00277d2200a7898a00a77e22003e
:10191800c7898a0016037800f1b79f00e2b79f00d5
:10192800d3b79f00c4b79f00b5b79f00060001005a
:1019380019007800e6c020008a03630087bf9f0073
:10194800a04390008ff39700274098004833de00ab
:10195800b043900036409800190078001e037800c4
:10196800804b9000064898004833de00904b90006a
:101978001648980019007800404390006ec0b300e4
:101988004e40980050439000584098001900780045
:10199800604390006c409800704390007b40980032
:1019a80019007800204b900028489800304b900090
:1019b80038489800190078000053900008509800a3
:1019c800105390001850980019007800404b900070
:1019d80048489800504b90005848980019007800e3
:1019e800604b900068489800704b900078489800c9
:1019f80019007800e63420008a03630087bf9f003f
:101a0800a05390008ff39700275098004833de00ca
:101a1800b05390003650980019007800005b900091
:101a280008589800105b9000185898001900780022
:101a380040539000485098005053900058509800d8
:101a480019007800605390006c5098007053900013
:101a58007b50980019007800205b90002858980067
:101a6800305b9000385898001900780000639000a7
:101a780008609800106390001860980019007800ba
:101a8800405b900048589800505b90005858980068
:101a980019007800605b90006c589800705b9000ab
:101aa8007b5898001900780020639000bfb2970017
:101ab80025609800b06290004fb29700346098009b
:101ac80019007800dfb197009301780000c29000f8
:101ad80003c09800c819de0010c2900013c0980017
:101ae800190078006fb1970012017800a0c190002a
:101af80022c098004811de00b0c1900032c09800a2
:101b08001900780040c1900048c0980050c190006a
:101b180058c098001900780060c1900068c098000b
:101b280070c1900078c098001900780042352000f4
:101b38008a01610000ca900003c898004811de00bd
:101b480090c9900012c8980019007800ffb097005b
:101b58009100780020c9900021c89800c808de00cc
:101b680030c9900031c898001900780021f22f0080
:101b7800898040000a81600080d1900002d09800de
:101b8800c808de0010d1900011d098001900780024
:101b9800c0d0900048d09800d0d0900058d098007d
:101ba80019007800e0d0900068d09800f0d090003c
:101bb80078d098001900780080d8900008d898004c
:101bc80090d8900018d8980019007800a0d89000f4
:101bd80028d89800b0d8900038d898001900780014
:101be800c0e0900048e09800d0e0900058e09800ed
:101bf80019007800e0e0900068e09800f0e09000bc
:101c080078e098001900780080e8900008e89800cb
:101c180090e8900018e8980019007800a0e8900073
:101c280028e89800b0e8900038e898009900780013
:101c3800114090000074a10090409800990078002d
:101c4800114090000054a10090409800990078003d
:101c5800114090000044a10090409800990078003d
:101c6800114090000064a00090409800190078008e
:101c78001004a100190078001014a1009900780040
:101c8800114090000034a10090409800ec8044007e
:101c98000080200080087800830f2000830e7800e1
:101ca800f0814400071420008709780072814400fd
:101cb8000090210000097800e486460000c3200057
:101cc800800e7800f484440040292500800c7800b8
:101cd8006a82400045d62100050a7800a5802200c6
:101ce800558a8a0005882200458a8a00858922004b
:101cf800658a8a0014027800f1b79f00e2b79f0056
:101d0800d3b79f00040001001900780004c1200027
:101d18008a02620020439000254098004822de0095
:101d2800b04290003440980019007800ffb0970046
:101d380091007800004a900001489800c808de0029
:101d4800104a90001148980019007800c04090008f
:101d58004e409800d04090005840980019007800f4
:101d6800e04090006c409800f04090007b40980064
:101d780019007800a048900028489800b0489000c2
:101d88003848980019007800805090000850980052
:101d9800905090001850980019007800c0489000a2
:101da80048489800d0489000584898001900780092
:101db800e048900068489800f048900078489800fb
:101dc80019007800013f20000a826000a0529000ac
:101dd80024509800c808de00305290003150980016
:101de8001900780080589000085898009058900082
:101df8001858980019007800c05090004850980072
:101e0800d05090005850980019007800e050900089
:101e18006c509800f05090007b50980019007800a2
:101e2800a058900028589800b0589000385898004a
:101e38001900780080609000086098009060900019
:101e48001860980019007800c05890004858980009
:101e5800d05890005858980019007800e058900021
:101e68006c589800f05890007b589800190078003a
:101e7800a0609000cfe0970021609800b0609000cb
:101e8800afe397003760980019007800dfb197003a
:101e98009300780080c1900001c09800c808de0057
:101ea80090c1900011c09800190078006fb1970098
:101eb8009200780020c1900021c09800c808de0078
:101ec80030c1900031c0980019007800c0c090005f
:101ed80048c09800d0c0900058c0980019007800f9
:101ee800e0c0900068c09800f0c0900078c09800ea
:101ef80019007800613f20000a81600080c99000c5
:101f080002c89800c808de0010c9900011c89800df
:101f1800190078009d00780020c9900021c8980019
:101f2800c808de0030c9900031c898001900780050
:101f380001f12f00898040000a85600000d19000df
:101f48000ad09800c808de0010d1900011d098007f
:101f580019007800c0d0900048d09800d0d09000e8
:101f680058d0980019007800e0d0900068d0980008
:101f7800f0d0900078d098001900780080d89000b0
:101f880008d8980090d8900018d8980019007800c0
:101f9800a0d8900028d89800b0d8900038d89800d9
:101fa80019007800c0e0900048e09800d0e0900068
:101fb80058e0980019007800e0e0900068e0980088
:101fc800f0e0900078e098001900780080e8900030
:101fd80008e8980090e8900018e898001900780040
:101fe800a0e8900028e89800b0e8900038e8980049
:101ff80099007800114090000074a100904098006a
:1020080099007800114090000054a1009040980079
:1020180099007800114090000044a1009040980079
:1020280099007800114090000064a000904098004a
:10203800190078001004a100190078001014a100fc
:1020480099007800114090000034a1009040980059
:102058007fa897004f0778004f06be004f05be00c7
:0c2068004f04be006f01b1000000060034
:020000040000fa
:102074000800fa00889fbe008a1f78008c1f780031
:102084001100200081bf9f008000eb0091bf9f00e2
:1020940091bf9f00101990009fb89700810f5100c5
:1020a4003b013600a6322000083620000604540006
:1020b4000884d100c7e1200005e020001fb9970083
:1020c400fe11b90082004000a1909000a1bf9f00c2
:1020d4001fb99700fe11b90082004000b190900032
:1020e400b1bf9f00bfb89700058153008191b9002b
:1020f400028142002fba97000402d0000482e90052
:1021040088a2b90084004300624290000482fb006c
:10211400f2419000c819dd00830172001fba9700d4
:10212400fe22b90004024000c49490001400200070
:102134008924dd008984ea0083846400e2419000fc
:102144008041eb0069419800c84cde007245900064
:1021540079419800624690000c86fb00724590001d
:102164004855dd000a0576001fbe9700fe66b900db
:102174008c044000d99490008924dd008984ea000d
:102184008a8464006245900069419800c84cde006e
:102194007245900079419800224690000c86fb001d
:1021a400324590004855dd000a0576001fbe9700b1
:1021b400fe66b9008c044000c99490008924dd00b7
:1021c4008984ea008a8464002245900029419800a9
:1021d400c84cde00324590003941980022469000f8
:1021e4000c86fb00324590004855dd000a05760058
:1021f4001fbe9700fe66b9008c044000d99490007d
:102204008924dd008984ea008a84640022459000e0
:1022140029419800c84cde003245900039419800ad
:10222400424e90000c86fb00524d90004855dd0054
:102234000a0576001fbe9700fe66b9008c044000b4
:10224400c99490008924dd0089047500424d9000f2
:1022540049499800c84cde00524d900059499800f5
:10226400424e90000c86fb00524d90004855dd0014
:102274000a0576001fbe9700fe66b9008c04400074
:10228400d99490008924dd0089047500424d9000a2
:1022940049499800c84cde00524d900059499800b5
:1022a400f0400a001188000021419000a3409800ea
:1022b40031419000b440980061419000e34098009f
:1022c4007141900002c3b300f240980001499000ac
:1022d4008348980011499000934898002149900040
:1022e40092c1b300a24898003149900092c0b30053
:1022f400b24898004149900002c4b300c248980013
:1023040051499000d448980021519000a35098005e
:1023140031519000b350980041519000c35098003f
:1023240051519000d350980061499000e3489800bf
:1023340071499000f348980001519000835098002f
:10234400115190009350980061519000e35098000f
:1023540071519000f35098000159900083589800ef
:10236400115990009358980021599000a35898004f
:1023740031599000b358980041599000c3589800bf
:1023840051599000d358980061599000e35898002f
:1023940071599000f35898000161900084c0b30013
:1023a4008460980011619000936098001fb99700b1
:1023b400fe11b90002014000c26c9100e1c4640046
:1023c40062002000824cdd00314190000264a100d3
:1023d40009417100b240980021619000a360980007
:1023e40031619000b36098001fb99700fe11b900e5
:1023f4000201400022999000c1649000c2609800dc
:102404004811de00d1649000d260980061619000b0
:10241400e360980071619000f36098001fb9970021
:10242400fe11b9000201400072919000816c90008d
:10243400826898004811de00916c900092689800c0
:1024440021699000a368980031699000b3689800ee
:1024540041699000c368980051699000d36898005e
:1024640061699000e368980071699000f3689800ce
:102474001fb99700fe11b900020140005299900063
:1024840081749000827098004811de00917490006d
:10249400927098001fb99700fe11b9000201400024
:1024a40042999000a1749000a27098004811de0037
:1024b400b1749000b27098001fb99700fe11b90072
:1024c4000201400062999000e15c9000e25898009b
:1024d4004811de00f15c9000f25898000161900010
:1024e4008460980011619000936098001fb9970070
:1024f4000200e0002c003a00314190000234a000b8
:10250400b2409800b141900082cfb30082c1610013
:102514000304a000b34098002142900003cfb3000d
:1025240083416200a3409800a149900002c1610068
:102534003240b300a24898001fb99700fe11b900b9
:102544000201400002999000e1699000e26898005d
:102554004811de00f1699000f26898007141900022
:102564000264a000f2409800414190000234a000af
:10257400c24098009fb897008100e80091bf9f0077
:10258400101990009fb89700810f5100cbfe3e00b8
:102594000fb897004f0678004f0578004f04be002f
:1025a4000080fa0000000600314190000234a100ce
:1025b400b24098003141900083cfb30003416100e1
:1025c4003240b300b24098002142900002cfb300e1
:1025d400024162000204a000a24098002149900038
:1025e40083416100a34898001fb99700fe11b90008
:1025f4000201400002999000e1699000e2689800ad
:102604004811de00f1699000f26898007141900071
:102614000264a000f2409800414190000234a000fe
:10262400c24098009fb897008100e80091bf9f00c6
:10263400101990009fb89700810f51009ffe3e0033
:04264400d3ff370089
:020000040000fa
:102648000600fa00889fbe008a1f7800100020004c
:10265800b0bf9f008000eb00c1bf9f000040eb00af
:10266800c0f79f00f08082000010a100f0808a006f
:10267800f08082000020a100f0808a00f0808200b3
:102688000030a100f0808a00f08082000040a100a4
:10269800f0808a00f08082000070a000f0808a003c
:1026a800f08082000090a100f0808a00f080820013
:1026b80000e0a000f0808a00f080820000f0a10015
:1026c800f0808a00000225000008eb0020002000ae
:1026d80050828a00820f200072828a0062bd200028
:1026e80062828a0080828a00c1bf9f008182820044
:1026f8004fb89700808f500009003600220525004a
:102708000009eb004fb897000000e800c0bf9f0029
:10271800818282004fb89700808f5000f8ff3e00fa
:10272800600525000008eb00640040000008eb008d
:102738000080e9000008eb00640040000008eb009e
:102748001000200010868a0020868a00e100200000
:1027580031868a00f100200041868a00a10c2500fc
:102768008048780009f4210069868a0008fa200068
:1027780078868a000314200093868a0083868a005c
:1027880005902100a5868a0082022000b2868a0070
:10279800c2868a00041e2000d4868a00f480400085
:1027a8008008eb00e0868a004100200001878a004b
:1027b80010878a006700200027878a0056002000bb
:1027c80036878a008a0e2500004d780059878a00ce
:1027d80068878a0083878a0073878a0095878a00ba
:1027e800a2878a00b2878a00c4878a0074014500dc
:1027f8000009eb00d0878a00760145000049eb000c
:102808006a0141000049eb00a3f62f0082814100d4
:1028180080497800c0f79f00b4c0b3000209b10036
:102828000449780082c0b30067824100024a7800f8
:1028380024c22000a4838a0068824100014a7800eb
:102848006b824100004aeb000482e900cff2970056
:10285800054a780000024200cff29700054a780046
:1028680063024200004aeb000402e900004aeb0060
:10287800f4ff270004848a0011848a00f282410050
:10288800800aeb0093417800e1c261008082620017
:10289800c92add00e37080000390a10083817200e3
:1028a800e370880065f72f008a824200804a78002a
:1028b800a3c0b30007844200034c78006784420039
:1028c800024c780008c2200008838a00688442000d
:1028d800014c78006b844200004ceb000884e9004e
:1028e800004ceb0000044400004ceb00630444007f
:1028f800004ceb000804e900004ceb0064838a00fc
:1029080071838a0007044400000ceb0095427800ac
:1029180061c46200000464004844dd00e570800082
:102928000580a10085027400e5708800e5f92f0094
:102938008a824200804a780007844200004c78006e
:1029480067844200004c7800e8c0200048848a0070
:1029580068844200014c7800eb8042008048eb001c
:10296800e98042008048eb00808040008048eb000e
:10297800e38040008048eb008100e9008048eb00dc
:10298800a4848a00b7848a0001802000c1848a0058
:102998009542780061c26200000262004222dd00b6
:1029a800e17080000120a10081007200e1708800c0
:1029b800ec0044008048780025c0b300720244004f
:1029c800054a780073024400024a780004c12000d6
:1029d800e4848a0074024400034a780077024400c1
:1029e800004aeb000482e900004aeb0000024200c2
:1029f800004aeb0063024200004aeb000402e900cf
:102a0800004aeb009140780061c260000002620059
:102a18004722dd00e17080000170a1008100720092
:102a2800e17088000102200088804000804878001a
:102a3800c0f79f0007824000064a7800678240007e
:102a4800024a780062c1200082858a0068814000bd
:102a5800034978006b8140000049eb000281e900de
:102a68000049eb00000141000049eb00630141000f
:102a78000049eb000201e9000049eb0091407800b1
:102a8800e1c0600000210a001c0e000081f62f0042
:102a9800828040008008eb00713e200021818a007e
:102aa8002209b1000009eb000281e9000009eb00ee
:102ab8007a0141000009eb0011828a0031002000f0
:102ac80031828a00318282000100e00001003a0070
:102ad80030828a00400425000008eb00400a2000ec
:102ae80040828a0050828200e20f50000d003200be
:102af800c00225000008eb00f07c200070818a00ed
:102b0800200325000008eb0060bd200080818a00ba
:102b18003fb897004f0578004f04be000080fa00c8
:102b2800000006000000eb00b0818a00703e200023
:102b3800c0818a0010002000e0818a00e1818200c3
:102b48000100e00001003a00e0818a00800f2000c7
:102b5800d0818a00c00225000008eb00f07c20002c
:102b680070818a00200325000008eb0060bd20006a
:102b780080818a003fb897004f0578004f04be0057
:0c2b88000080fa0000000600e6ff3700a5
:020000040000fa
:102b94000400fa00889fbe008a1f780000047800b1
:102ba4000000eb00c0bf9f00800478000800e00034
:102bb400350032001800e00038003d002800900085
:102bc4008004eb000000e0002f0032003800900089
:102bd4000000e0002c003200480090000000e000fb
:102be40029003200580090000000e0002600320066
:102bf4001838a30035003a003c62ab0022003a00ca
:102c04003c22ab0044003a00190020003e22ab00f5
:102c14001d003a0020128000e0f79f0011800a0096
:102c2400180000000004e00043003a0011c4b3009f
:102c34006ff19700814f51007600320030c4b30029
:102c4400eff0970080cf5000bb003200b0c4b30057
:102c54006ff19700804f5100c80032001900200026
:102c640040c5b300eff0970080cf500006003a0053
:102c74006ff19700425c98001810a0002914980086
:102c84002000200010049800090078004f05780007
:102c94004f04be000080fa000000060029149800ca
:102ca4001810a1001800a1001830a1001820a100dc
:102cb40019002000090078004f0578004f04be0079
:102cc4000080fa0000000600f4ff3700190020001d
:102cd4003ce2ab00ecff320028109000890f50005a
:102ce400e9ff3a0080002000c0bf9f004fb8970062
:102cf400ef0f50000b003e004fb897000000440057
:102d0400404890000080fb00401288004fb89700b4
:102d14000000e800f4ff37003c22a900190020005d
:102d2400e4ff37001830a1000000eb0020149800e5
:102d340019002000dfff3700281090000000440035
:102d4400eff0970041589800281090000000e80028
:102d5400201498002810900019002000e30f500060
:102d6400c9ff36001810a1000005eb002a149800d2
:102d740000302500ca0b0700886090007858900046
:102d840080cf5000c0ff3a0058589000e858900097
:102d9400c808dd000080fb0000804000101498008b
:102da40048599000424c980018109000504c9800dc
:102db400181090004800de00604c980000c3b30077
:102dc400704c98000054980010c6b300105498003a
:102dd40000c0e80020549800684040003054980037
:102de400cabf9f004fb89700e70f50004b003e004a
:102df4004fb8970000004400404890000080fb005a
:102e0400401288004fb897000000e800c0bf9f0040
:102e1400f4ff3700a800900091007800414c98001e
:102e2400a800900091007800c808de00514c98007a
:102e3400b800900091007800614c9800b8009000b0
:102e440091007800c808de00714c9800c80090001a
:102e54009100780001549800c80090009100780017
:102e6400c808de0011549800d80090009100780042
:102e740021549800d800900091007800c808de0022
:102e8400315498004054980050549800605498006d
:102e940070549800005c9800105c9800205c9800c6
:102ea400305c98001830a000291498000000eb0052
:102eb400c0bf9f004fb89700e70f500072ff3e005d
:102ec4004fb8970000004400404890000080fb0089
:102ed400401288004fb897000000e800c0bf9f0070
:102ee4004fb89700e70f500071ff3e004fb89700ae
:102ef40000004400404890000080fb00401288001d
:102f04004fb897000000e800c0bf9f004fb897007b
:102f1400e70f5000eaff360065ff37001800900005
:102f2400e20f500062ff3a001814900068828a0091
:102f3400190020005fff370060072000401288005e
:102f44004822ef004822ef001900200049128800af
:102f54004822ef004822ef004822ef000900400019
:102f640040128800090078004f0578004f04be0025
:102f74000080fa000000060048ff37006ff0970059
:102f8400405c98001810a000190020002914980033
:0c2f94000000eb00100498003bff370029
:020000040000fa
:102fa0000400fa000002780011002000f1bf9f0029
:102fb0001404e00048003200e4409000efcf5000dd
:102fc00049003e0054499000e44090000281fb001b
:102fd0008180fb008110dd0001007800d02bb7005c
:102fe00024499000e44090000281fb008180fb00b6
:102ff0008110dd0001007800f02bb700144990002b
:10300000e44090000281fb008180fb008110dd0024
:1030100001007800202bb700e4409000e7cf50007b
:1030200050003e00e440900081c04000c1ff9f007e
:10303000e440900002b1200012417800c4489000a2
:103040008180fb004ff897008081fb008308dd0042
:103050008140710002b120000149780002b12000d6
:1030600012417800b44990008381fb004ff897002b
:103070008080fb008100e8008118dd008140710044
:1030800002b1200001497800e44090008180fb00fb
:1030900002b82000828040000449900082487800f5
:1030a000f4409000e1cf500057003200e1cf5000d3
:1030b0005c003900e2cf50006b003200e3cf5000db
:1030c000620032008af0a800344890000004e0005a
:1030d000010032008cf0a800ffb8970001007800d2
:1030e0000080fa0000000600644190008000eb00c0
:1030f000ff4f5100f9ff3e0054499000e44090001a
:103100000281fb008180fb00f08050008110dd0017
:1031100001007800d22bb70024499000e4409000d1
:103120000281fb008180fb00f08050008110dd00f7
:1031300001007800f22bb70014499000e4409000a1
:103140000281fb008180fb00f08050008110dd00d7
:1031500001007800222bb700e4409000e7cf500038
:10316000b0ff3600e4409000efcf5000340036004e
:10317000e4409000f7cf500042003e00e440900051
:10318000f0c0500081c04000c1ff9f00e4409000ab
:1031900002b1200012417800c44890008180fb00f9
:1031a0004ff897008081fb008308dd0081407100ab
:1031b00002b120000149780002b1200012417800dc
:1031c000b44990008381fb004ff897008080fb009a
:1031d0008100e8008118dd008140710002b120000b
:1031e00001497800e44090008180fb0002b8200093
:1031f000828040000449900082487800f4409000aa
:10320000e1cf5000a9ff3a008a30a800344890006e
:103210000004e000b0ff32008c30a800ffb8970037
:10322000aeff37008a10a800344890000004e00088
:10323000a9ff32008c10a800ffb89700a7ff370045
:10324000e4409000e8c0500077ff37008a70a80083
:10325000344890000004e0009fff32008c70a8000a
:10326000ffb897009dff37008a50a80034489000af
:103270000004e00098ff32008c50a800ffb89700cf
:1032800096ff3700644190008000eb00ff4f510033
:1032900092ff3e00e4409000f8c0500062ff37000b
:020000040000fa
:1032a0000200fa00881f7800000478000000eb009c
:1032b000e0bf9f00f0000a00180000004004210059
:1032c000c860900040649800c800de00586190001b
:1032d00051649800e80040006861900061649800c3
:1032e000c808de0078619000716498000100250034
:1032f00008699000016c9800c808de001869900009
:10330000116c98004100250028699000216c9800fc
:10331000c808de0038699000316c98009180800008
:103320006871900061749800c808de0078719000a0
:1033300071749800a180800008799000017c980049
:10334000c808de0018799000117c98007184800014
:1033500028799000217c9800c808de003879900018
:10336000317c980081808000487190004174980001
:10337000c808de00587190005174980001808000e8
:1033800048699000416c9800c808de0058699000b8
:10339000516c98001180800068699000616c980001
:1033a000c808de0078699000716c98002180800068
:1033b0000871900001749800c808de001871900030
:1033c0001174980031808000287190002174980059
:1033d000c808de0038719000317498008000eb005e
:1033e000e1bf9f00486990000281fb00d86890000f
:1033f000c808dd00810071006fb99700828f50000e
:103400001c003600810021006fb99700efb99700ca
:10341000c219dd00838140004211dd00020140003d
:1034200033197800231178006fb99700efb997002e
:10343000c219dd00838140004211dd00020140001d
:103440003319780023117800efb997008301e80061
:10345000e3bf9f00c86990008381fb00586990001a
:103460004811dd0002817100efb99700830f510010
:10347000e5ff3e008000eb00e1bf9f00686990001f
:103480000281fb00f8689000c808dd00810071002f
:103490006fb99700828f500027003600c133250096
:1034a0006fb99700efb99700c219dd008381400022
:1034b0000281e8004211dd0002014000331978006a
:1034c000231178006fb99700efb99700c219dd009a
:1034d000838140000281e8004211dd0002014000ca
:1034e00033197800231178006fb99700efb997006e
:1034f000c219dd00838140000281e8004211dd0035
:10350000020140003319780023117800efb99700c9
:103510008301e800e3bf9f00e86990008381fb001e
:10352000786990004811dd0002817100efb99700c1
:10353000830f5100daff3e00c01b25002c0407005a
:10354000b0808000e8789000607c98004800de0041
:10355000f8789000707c980080848000c878900093
:10356000407c98004800de00d8789000507c98009d
:10357000100020004f0478000080fa0000000600d0
:020000040000fa
:103580000400fa0012002000e2bf9f008000eb0060
:10359000f1bf9f000000e000200032001000e000ba
:1035a00021003d00100190008000eb000200e000cf
:1035b0001a0032009000900011017800d0009000b5
:1035c00081006100f1bf9f00a00090000100e000b9
:1035d00007003200900090009100780020019000d8
:1035e0009280500001f0a7008100ea00f1bf9f0027
:1035f000a8810a0010000000e38f50005b00320039
:1036000010003400e58f5000760032006b0035006a
:10361000e68f50002f0032008000eb0001007800a0
:103620000080fa0000000600610098001010a10060
:103630001000a100020078000080fa0000000600df
:10364000f9ff3700e18f500052003200e28f500046
:10365000f1ff3a0070019000ffb89700810f510010
:103660006a0036001010a0001018a30024003200d9
:1036700010017800e10061000104e00020003a0040
:10368000e00090008100e800610098006001900077
:1036900080089000810f5100090039001000a0003f
:1036a0008008900061009800b00090000100e000e8
:1036b000030032003000900000000100e0bf9f00d6
:1036c000efb89700010078000080fa0000000600c3
:1036d000d5ff370010099000ffb89700810f510007
:1036e000e0ff3e0070019000ffb89700810f51008d
:1036f000dcff39001010a1001018a300dcff3a0015
:1037000010017800e10061000104e00013003200c4
:103710001018a30011003a00e00090008100e800ba
:103720006100980060019000a0089000810f510096
:10373000e3ff39001000a100a0089000610098008c
:10374000c00090000100e000ddff3200400090006a
:1037500000000100e0bf9f00d9ff37008000eb00b0
:1037600061009800efb89700d6ff37007001900015
:10377000ffb89700810f5100baff3200700190002e
:10378000ffb89700810f5100b7ff32001010a10061
:10379000d9ff370070019000ffb89700810f5100ea
:1037a000b0ff390010099000ffb89700810f510059
:1037b000adff36001010a100cfff37007001900060
:1037c000ffb89700810f5100a6ff3a0070019000ea
:1037d000ffb89700810f5100a3ff3a001010a1001d
:1037e000c5ff370010099000ffb89700810f510006
:1037f000c0ff310070019000ffb89700810f5100a9
:10380000bcff36001010a00097ff37001009900091
:10381000ffb89700810f510093ff31001010a100f5
:04382000b5ff3700b9
:020000040000fa
:103824000200fa008000eb00f1bf9f00f0010a00e3
:103834001000000081052100406190004160980063
:103844004809de00d0619000526098006881400011
:10385400e0619000626098004811de00f061900021
:1038640072609800a20025008069900002689800a8
:103874004811de009069900012689800e20025006b
:10388400a0699000226898004811de00b069900099
:103894003268980052818000e07190006270980054
:1038a4004811de00f071900072709800628180000f
:1038b40080799000027898004811de009079900099
:1038c4001278980092848000a07990002278980061
:1038d4004811de00b079900032789800428180006f
:1038e400c0719000427098004811de00d0719000c1
:1038f40052709800c2808000c069900042689800ad
:103904004811de00d069900052689800d28080008f
:10391400e0699000626898004811de00f069900048
:1039240072689800e28080008071900002709800b4
:103934004811de009071900012709800f2808000af
:10394400a0719000227098004811de00b0719000c0
:10395400327098000001eb00f2bf9f00c069900034
:103964008381fb00506990004811dd0002817100e1
:10397400ffb99700830f51001c003600020221009a
:10398400ffb997007fba97004222dd00040241008c
:10399400c219dd0083814000b4197800a4117800b5
:1039a400ffb997007fba97004222dd00040241006c
:1039b400c219dd0083814000b4197800a411780095
:1039c4007fba97000402e800f4bf9f00406a9000a9
:1039d4000482fb00d0699000c819dd0083017200e5
:1039e4007fba9700848f5100e5ff3e000001eb0091
:1039f400f2bf9f00e06990008381fb007069900032
:103a04004811dd0002817100ffb99700830f510056
:103a14002700360082342500ffb997007fba97004b
:103a24004222dd00040241008381e800c219dd0066
:103a340083814000b4197800a4117800ffb997007d
:103a44007fba97004222dd00040241008381e8002e
:103a5400c219dd0083814000b4197800a4117800f4
:103a6400ffb997007fba97004222dd0004024100ab
:103a74008381e800c219dd0083814000b419780015
:103a8400a41178007fba97000402e800f4bf9f00f5
:103a9400606a90000482fb00f0699000c819dd00a0
:103aa400830172007fba9700848f5100daff3e00d1
:103ab400802225003a050700100020000080fa004b
:043ac40000000600f8
:020000040000fa
:103ac8000200fa008000eb00f1bf9f00f0010a003d
:103ad80010000000c106210040619000416098007c
:103ae8004809de00d061900052609800688140006b
:103af800e0619000626098004811de00f06190007b
:103b08007260980042012500806990000268980060
:103b18004811de0090699000126898008201250023
:103b2800a0699000226898004811de00b0699000f2
:103b38003268980002828000e071900062709800fc
:103b48004811de00f07190007270980012828000b7
:103b580080799000027898004811de0090799000f2
:103b680012789800a2848000a079900022789800aa
:103b78004811de00b079900032789800f281800018
:103b8800c0719000427098004811de00d07190001a
:103b98005270980072818000c06990004268980055
:103ba8004811de00d0699000526898008281800038
:103bb800e0699000626898004811de00f0699000a2
:103bc800726898009281800080719000027098005d
:103bd8004811de009071900012709800a281800058
:103be800a0719000227098004811de00b07190001a
:103bf800327098000001eb00f2bf9f00c06990008e
:103c08008381fb00506990004811dd00028171003a
:103c1800ffb99700830f51001c0036006203210092
:103c2800ffb997007fba97004222dd0004024100e5
:103c3800c219dd0083814000b4197800a41178000e
:103c4800ffb997007fba97004222dd0004024100c5
:103c5800c219dd0083814000b4197800a4117800ee
:103c68007fba97000402e800f4bf9f00406a900002
:103c78000482fb00d0699000c819dd00830172003e
:103c88007fba9700848f5100e5ff3e000001eb00ea
:103c9800f2bf9f00e06990008381fb00706990008b
:103ca8004811dd0002817100ffb99700830f5100b0
:103cb8002700360042352500ffb997007fba9700e4
:103cc8004222dd00040241008381e800c219dd00c0
:103cd80083814000b4197800a4117800ffb99700d7
:103ce8007fba97004222dd00040241008381e80088
:103cf800c219dd0083814000b4197800a41178004e
:103d0800ffb997007fba97004222dd000402410004
:103d18008381e800c219dd0083814000b41978006e
:103d2800a41178007fba97000402e800f4bf9f004e
:103d3800606a90000482fb00f0699000c819dd00f9
:103d4800830172007fba9700848f5100daff3e002a
:103d580040292500e8040700100020000080fa0030
:043d68000000060051
:020000040000fa
:103d6c000600fa0010002000d0bf9f000000eb00fe
:103d7c00e0bf9f00f0bf9f0011618000d1828a00dc
:103d8c007160800091828a0081608000a1828a002b
:103d9c00b1608000e1828a00e0bf9f0081828200d6
:103dac006fb89700808f500010003600e20125009c
:103dbc006fb897007a0040000000400000004100fe
:103dcc00900078007fb8970000804000f0bf9f0003
:103ddc006fb897000000e800e0bf9f00818282006e
:103dec006fb89700808f5000f1ff3e007fb89700ae
:103dfc00b0828a00d28282000000eb00612b20008e
:103e0c00810f510005003600d28282001000200084
:103e1c00113f2000810f510024003e006100600022
:103e2c00c300dd00f08082000030a1000080700033
:103e3c00f0808a00748a8200208b8200d38b8200ef
:103e4c00828c8200318d82000400700003007000af
:103e5c000200700081007000e1806000c708dd0086
:103e6c00f08082000070a10000807000f0808a0059
:103e7c00e001250080f20700dfb897000100600028
:103e8c00d0bf9f007e05070000818200e40f500028
:103e9c0025003e00d08b820000f0a100d08b8a0060
:103eac005fb897000080fa00000006000000eb00ed
:103ebc0061006000c300dd00f08082000030a100d2
:103ecc0000807000f0808a00748a8200208b82004f
:103edc00d38b8200828c8200318d820004007000b2
:103eec00030070000200700081007000e18060002f
:103efc00c708dd00f08082000070a1000080700017
:103f0c00f0808a00e00125005bf20700dfb8970023
:103f1c0001006000d0bf9f0059050700008182009e
:103f2c00e40f5000dbff3600e0888200a0609000b8
:103f3c008180fb00306090004800dd000080700044
:103f4c00f08b8a00e08882009040900077810a0014
:103f5c0001000000cf08dd00d08b820000f0a10032
:103f6c0000807000d08b8a005fb897000080fa0048
:083f7c0000000600cdff370034
:020000040000fa
:103f84000200fa000000eb00f0bf9f0000002700d1
:103f9400840fb60021003200a10920008007200010
:103fa4000001eb0053f82000804978008149780033
:103fb40082497800207c8000e007b2000000a00065
:103fc400720520006104200043f820008149780034
:103fd4008249780080497800eca10a00840f00002f
:103fe400a8a00a00840f000080cf50000600320011
:103ff4007fb897008000e800f1bf9f00713821006e
:10400400810f5000f4ff36000000eb0071382100ee
:104014007fb99700810f51003b003e0000fc2f0048
:104024008c2fb600860fb6000000a000307c8800fc
:10403400800c2000b0200a00880f0000f0f82f0048
:104044008a0fb6000060a000507c880080ff2f001b
:104054008a0fb6000000a000507c8800f0cf2f002b
:104064008a2fb600a109200012002000800720003a
:1040740053f820008049780081497800824978000b
:10408400eca10a00840f0000a8a00a00840f00001d
:1040940080cf500022003200207c8000e007b20074
:1040a4000000a000720520006104200043f82000f5
:1040b400814978008249780080497800eca10a009f
:1040c400840f0000a8a00a00840f000080cf5000d5
:1040d400060032007fb897008000e800f1bf9f001f
:1040e40071382100810f5000f4ff3600eca20a0061
:1040f400840f0000a8a10a00840f00000000eb0058
:10410400814f5100020032000080fa0000000600d6
:10411400713821007fb99700810f5100faff3e00ea
:1041240084efa80084afab0006003a007fb8970084
:104134008000e800f1bf9f0071382100810f50001a
:10414400f8ff36000000eb0084afab00eeff320056
:10415400713821007fb99700810f5100eaff3e00ba
:1041640033a00a00840f0000610010000080fa00f0
:0841740000000600e6ff370021
:020000040000fa
:10417c000200fa0011002000f1bf9f00a52fa9003a
:10418c002be3a90061e3a90097e3a900cde3a90003
:10419c0003e4a90039e4a9006fe4a900a5e4a9008f
:1041ac0031002000f0210a00000300002130200023
:1041bc00914078000263ef0031302000914078008c
:1041cc000363ef0041302000914078000463ef005e
:1041dc0051302000914078000563ef0061302000e1
:1041ec00914078000663ef00713020009140780018
:1041fc000763ef0081302000914078000863ef00e6
:10420c0091302000914078000963ef00a13020002c
:10421c00914078000a63ef00b130200091407800a3
:10422c000b63ef00c06891000104e000080032004d
:10423c0070909000a1302000914078000ae3b70004
:10424c004800de00b1302000914078000be3b7004d
:10425c000cc3bf000c63ef000dc3bf000d63ef0078
:10426c000ec3bf000e63ef000fc3bf000f63ef0060
:10427c0010c3bf001063ef0011c3bf001163ef0048
:10428c0012c3bf001263ef0013c3bf001363ef0030
:10429c0014c3bf001463ef0015c3bf001563ef0018
:1042ac0016c3bf001663ef0017c3bf001763ef0000
:1042bc0018c3bf001863ef0019c3bf001963ef00e8
:1042cc001ac3bf001a63ef001bc3bf001b63ef00d0
:1042dc001cc3bf001c63ef001dc3bf001d63ef00b8
:1042ec001ec3bf001e63ef001fc3bf001f63ef00a0
:1042fc0020c3bf002063ef0021c3bf002163ef0088
:10430c0022c3bf002263ef0023c3bf002363ef006f
:10431c0024c3bf002463ef0025c3bf002563ef0057
:10432c0026c3bf002663ef0027c3bf002763ef003f
:10433c0028c3bf002863ef0029c3bf002963ef0027
:0c434c007fb897000080fa000000060017
:020000040000fa
:10435800889fbe00a9052500898a8a008000eb0095
:10436800918a8a008082eb00c58a8a00e7142500ba
:10437800f48f2f00170062000090a000800b7800d7
:10438800d18a8a00602b2000e08a8a002603200058
:10439800f68a8a00502f2000008b8a00481f2000d0
:1043a800188b8a0043e72200a38a8a00c2ed220004
:1043b800b28a8a00401625001010a0001000a00044
:1043c80017f0a000398b8a00418b8a00758b8a0010
:1043d800900362000780a00007087800818b8a009c
:1043e800273f2000978b8a00a68b8a00373b200046
:1043f800b78b8a00c88b8a00538b8a00628b8a002d
:104408001010a0001000a00010f0a0000980e90022
:10441800e08b8a006e805400f08b8a00258c8a001d
:10442800a0172500900362000780a0000708780005
:10443800318c8a00e7072000478c8a00a70f2000ec
:10444800578c8a00f7012000678c8a00873e20007d
:10445800778c8a00038c8a00128c8a001010a100c5
:104468001000a10010f0a10064805400908c8a0014
:10447800a18c8a00d58c8a0000192500900362005f
:104488000780a00007087800e18c8a00f7942100d3
:10449800f78c8a00068d8a00a720b100178d8a0044
:1044a800077d2000278d8a00b38c8a00c28c8a0081
:1044b8001010a0001000a00010f0a0000980e80073
:1044c800408d8a00518d8a00858d8a00601a2500ea
:1044d800100262000480a00004087800918d8a0010
:1044e80051632000a18d8a00b68d8a001104b100a5
:1044f800c18d8a00d78d8a00638d8a00728d8a00eb
:104508001010a0001000a00010f0a0001000200063
:084518004f04be000000060084
:020000040000fa
:1045200010f0a6002d0037002014900040159000d8
:104530008608c3008608c1001201c100301b90002c
:104540000600c8001a039000260598000a03900090
:104550001605980010019000920078000029900044
:10456000010978001011900092801000201990002d
:104570008208dd0030149000010d78008688c300a9
:104580008688c1008688c1001281c100401b90004e
:104590000680c8000000cb000400cd00102390006e
:1045a00016a0e60006027800002390001620e60020
:1045b00006027800100c9000040c7800500c90005b
:1045c000040c7800401590000a039000160598002e
:1045d000040d7800f6220400000000001001900095
:1045e0009200780000299000010978000000060080
:1045f000801f7800401090000018eb000008eb00ce
:104600004f007800801f7800501090000018eb00d9
:104610000018eb000008eb004f00780000000600d7
:10462000801f7800811f78005010900001187800da
:104630000118780001087800cf0078004f0078005a
:10464000801f7800821f78004010900002187800c8
:10465000020878004f0178004f0078000000060043
:1046600010f0a6001a0037001001900092007800a8
:10467000002990000109780010119000928010002c
:10468000201990008208dd00701b900060199000d6
:10469000010278001301c1000200c8000400cd002f
:1046a0001023900016a0e600060278000023900078
:1046b0001620e60006027800100c9000040c78002a
:1046c000500c9000040c78007023040000000000df
:1046d00010019000920078000029900001097800f4
:0446e00000000600d0
:020000040000fa
:1046e4004e5100006e000000800000001e500000cb
:1046f4003001000080000000801000000a0000006b
:10470400800000000053000026000000800000002c
:104714008a10000004000000800000003c530000e8
:104724000c00000082000000334d0000007c0000fb
:1047340000004a00b3000000bc5100006c000000ff
:10474400800000000010000018000000820000003b
:1047540002000300000200000300c4005100000036
:104764003dee000000030000ffff030000d65400ec
:104774008e100000040000008000000044100000bf
:104784001400000080000000005000000a00000037
:1047940080000000485300000c000000820000006c
:1047a4007a420000000d040000009300c1000000e4
:1047b400285200006c000000800000001810000067
:1047c4001600000082000000020003000002000046
:1047d4000300e600410000001bfe0000000500008d
:1047e400ffff04000000000092100000020000001f
:1047f4008000000058100000140000008000000039
:104804000a5000000a000000800000005453000019
:104814000c000000820000007a420000000d040039
:1048240000009300c1000000945200006c000000de
:10483400800000002e10000016000000820000001e
:1048440002000300000200000300e6004100000033
:104854001bfe000000050000ffff04000000000034
:104864009410000002000000800000006c100000a2
:104874001400000080000000145000000a00000032
:084884008000000000000000ac
:020000040000fa
:10488c000800fa0011002000c1bf9f008000eb005f
:10489c00d1bf9f00e1bf9f00f1bf9f00d1bf9f0020
:1048ac0010199000dfb89700810f510056003600a8
:1048bc00a432200005362000848252008582d1006b
:1048cc005fb99700fe11b90082004000a1909000e2
:1048dc00f1bf9f007fb997000201d0000281e9006f
:1048ec008591b90082004200e14190008381fb0078
:1048fc00714190004811dd0002817100030023001a
:10490c0002817100e1419000e24098004811de0004
:10491c00f1419000f2409800814990008381fb00a6
:10492c00114990004811dd0002817100820178006c
:10493c00330fb200014b9000834898004811de0001
:10494c009149900092489800114190000274a00087
:10495c0092409800414190000234a000c24098005f
:10496c001181fb00914190000278a3000e003200ef
:10497c000003e200060035006fb997008201e800e1
:10498c00e3bf9f0073382100830f5100f8ff3600fe
:10499c00efb9970072382100828f51001d003e0044
:1049ac0001c3ab001b003a00814990008381fb00de
:1049bc00114990004811dd0002817100c200b30062
:1049cc0081499000824898004811de00914990007e
:1049dc00924898009140900077810a0001000000f5
:1049ec004fb9970082806000c1bf9f00dfb897006d
:1049fc008100e800d1bf9f0010199000dfb897002c
:104a0c00810f5100aeff3e004fb897000080fa00b6
:104a1c00000006000000eb000080fa000000060019
:044a2c00fcff370054
:020000040000fa
:104a30000200fa0012002000f2bf9f0090029000d6
:104a400003e02000c4e120000302520085a2b90067
:104a500083004200b00190000300e0002e003a0005
:104a6000614290000482fb00f1419000c819dd0012
:104a700083017200200290000411dd000281ea002f
:104a800003016100e1419000e24098004811de001e
:104a9000f1419000f2409800400190000200e000d7
:104aa0002d003200214290000482fb00b1419000b1
:104ab000c819dd008301720020019000140020005d
:104ac0000221dd0002817100a1419000a240980006
:104ad0004811de00b1419000b24098001182fb0005
:104ae00091419000c819dd008301720020019000ff
:104af000100020000201dd000281ea0003016100d4
:104b0000f0020a0011000000f0bf9f007fb897007c
:104b10000080fa0000000600614290000482fb0061
:104b2000f1419000c819dd0083017200200290005d
:104b30000411dd0002817100e1419000e240980023
:104b40004811de00f1419000f240980040019000d1
:104b50000200e000d3ff3a00214290000482fb00f3
:104b6000b1419000c819dd0083017200200190005e
:104b7000140020000221dd000281ea00030161002f
:104b8000a1419000a24098004811de00b141900080
:104b9000b24098001182fb0091419000c819dd00dd
:104ba0008301720020019000100020000201dd004e
:104bb0000281ea0003016100f0020a001100000016
:104bc000f0bf9f007fb897000080fa000000060049
:044bd000d1ff3700da
:020000040000fa
:104bd4000600fa0011002000d1bf9f008000eb0006
:104be400e1bf9f00f1bf9f00e1bf9f00101990003b
:104bf400efb89700810f510051003600a332200016
:104c040004362000030252000482d1006fb99700d9
:104c1400fe11b90082004000a1909000f1bf9f00f6
:104c24007fb997000201d0000281e9008491b900a4
:104c340082804100e14290008582fb007141900036
:104c44004811dd0002817200050023000281720018
:104c5400e1429000e24098004811de00f1429000e9
:104c6400f2409800814a90008582fb00114990002f
:104c74004811dd000281720082027800350fb20013
:104c8400014b9000854898004811de00914a90003d
:104c9400924898009182fb00114190004811dd0078
:104ca4000281720002f0a100f0020a00110000006b
:104cb4006fb99700fe11b9000201400022999000db
:104cc400c1629000c26098004811de00d162900079
:104cd400d2609800c14290008582fb00514190004f
:104ce4004811dd00028172000230a000c142900030
:104cf400c24098004811de00d1429000d240980092
:104d04001141900001c8b300814061008180fb0023
:104d14008100e900cf08de005fb99700828060005f
:104d2400d1bf9f00efb897008100e800e1bf9f006a
:104d340010199000efb89700810f5100b3ff3e00a7
:0c4d44005fb897000080fa000000060035
:020000040000fa
:104d50000200fa0010002000f0bf9f00a40fa9007d
:104d600001eba90001aba90000062000022bb7004f
:104d700002eba90005eba90005cba900058ba80053
:104d800000702000042bb70003f82f00205880008b
:104d9000808061000110a00021588800a10020003f
:104da00090210a00060b000007cba90007eba90021
:104db000f1ff210082b0200012896000098ba90058
:104dc000096ba900094ba900092ba900090ba9002f
:104dd00008eba90008cba90001fc2f0080b020003f
:104de00010886000f1ff230052588000828060002c
:104df00001f0a00051588800f10f2c00a0b0200055
:104e0000108860000aeba9000a0ba9000a2ba90070
:104e10000c0ba9000c2ba900c1ff2f00e2b0200051
:104e20001289600031ff2f00e0b020001088600080
:104e300000eca900000ca900002ca90000f0200043
:104e4000022cb70002eca900020ca900022ca90058
:104e50008000eb0090210a00d80b000090210a008e
:104e6000d40b00000230200002007800d62bb700df
:104e7000b05e8000808061000110a000b15e8800fb
:104e800001c0210001007800d62bb7000200780095
:104e9000da2bb700d25e8000028061000010a00013
:104ea000d05e880001007800da2bb7007fb8970049
:084eb0000080fa00000006007a
:020000040000fa
:104eb80010f0a60034003700201490004015900030
:104ec8008608c3008608c1001201c100301b90008b
:104ed8000600c8001a039000260598000a039000ef
:104ee80016059800100190009200780000299000a3
:104ef80001097800400190008100110010e0a7002e
:104f08008100ea0010119000928010002019900092
:104f18008208dd0030149000010d78008688c300f7
:104f28008688c1008688c1001281c100401b90009c
:104f38000680c8000000cb000400cd0010239000bc
:104f480016a0e60006027800002390001620e6006e
:104f580006027800100c9000040c780041a3de00d3
:104f68005024900008054300402490000a0c780063
:104f7800401590000a03900016059800040d78006b
:104f8800d027040000000000100190009200780073
:104f9800002990000109780000000600801f7800b1
:104fa800401090000018eb000008eb004f0078005c
:104fb800801f7800501090000018eb000018eb00dc
:104fc8000008eb004f00780000000600801f780002
:104fd800811f78005010900001187800011878009f
:104fe80001087800cf0078004f007800801f780013
:104ff800821f78004010900002187800020878009c
:105008004f0178004f0078000000060010f0a6005d
:105018003400370020149000401590008608c30023
:105028008608c1001201c100301b90000600c800ac
:105038001a039000260598000a03900016059800a8
:105048001001900092007800002990000109780072
:10505800400190008100110010e0a7008100ea00e3
:105068001011900092801000201990008208dd0035
:1050780030149000010d78008688c3008688c1002e
:105088008688c1001281c100401b90000680c800bc
:105098000000cb000400cd001023900016a0e6000d
:1050a80006027800002390001620e6000602780029
:1050b800100c9000040c780041a3de0050249000ee
:1050c80008054300402490000a0c78004015900021
:1050d8000a03900016059800040d78007e28040045
:1050e8000000000010019000920078000029900054
:1050f8000109780000000600801f78004010900029
:105108000018eb000008eb004f007800801f7800c3
:10511800501090000018eb000018eb000008eb009e
:105128004f00780000000600801f7800811f78007b
:1051380050109000011878000118780001087800d4
:10514800cf0078004f007800801f7800821f780019
:105158004010900002187800020878004f0178008b
:085168004f0078000000060072
:020000040000fa
:105170000600fa0011002000d1bf9f008000eb0064
:10518000e1bf9f00e1bf9f0010199000efb89700aa
:10519000810f51003c003600a53220000636200069
:1051a000050353000683d1006fb99700fe11b900c3
:1051b00082004000a1909000f1bf9f007fb997004e
:1051c0000201d0000281e9008691b900828042008c
:1051d000614190000281fb00714290004822dd0095
:1051e00004027100030023000482710061419000f9
:1051f0000041eb00e44098004822de00f1439000bb
:10520000f440980041629000c260980051629000a2
:10521000d2609800414290000482fb00514190000e
:105220004811dd00020172000230a00041429000ee
:10523000c24098004811de0051429000d2409800d0
:10524000614190000281fb00f1409000c808dd0040
:1052500081007100838160008301ea00cf19de00c4
:10526000dfb8970081816100d3bf9f00efb897003e
:105270008100e800e1bf9f0010199000efb897008f
:10528000810f5100c8ff3e005fb897000080fa0010
:045290000000060014
:020000040000fa
:105294000400fa0010002000e0bf9f000000eb00b3
:1052a400f0bf9f0036fb0700efb8970001006000d5
:1052b400e0bf9f00c2010700efb897000100600043
:1052c400e0bf9f0062020700efb897000100600092
:1052d400e0bf9f00a3000700efb897000100600043
:1052e400e0bf9f003f020700efb897000100600095
:1052f400e0bf9f005d010700efb897000100600068
:10530400e0bf9f0013fc0700efb8970001006000a6
:10531400e0bf9f0083020700efb897000100600020
:10532400e0bf9f00f0f82f004028b6000028a90035
:105334002028a90001e1a800000880004f00de0039
:10534400efb8970001006000e0bf9f006fb89700be
:105354000000e00001003a000000fe000028ab005d
:1053640006003a007fb897008000e800f1bf9f0074
:10537400f1522700810f5000f8ff36000028a900e1
:105384000000eb00f0bf9f0077fa0700f60107006a
:0c5394007302070000000000f0ff37006b
:020000040000fa
:1053a0000600fa0011002000d1bf9f008000eb0032
:1053b000e1bf9f00f1bf9f00e1bf9f001019900067
:1053c000efb89700810f51002d003600a432200065
:1053d00005362000848252008582d1006fb9970083
:1053e000fe11b90082004000a1909000f1bf9f0023
:1053f0007fb997000201d0000281e9008591b900d0
:1054000082004200414190000234a000c240980056
:10541000614190000281fb00f1419000c819dd005c
:10542000830171004819de0061439000e340980059
:10543000f20cb200f1419000f240980061419000fe
:10544000f1409000c808dd00020023008280600067
:105450008100e900cf08de005fb99700828060001c
:10546000d1bf9f00efb897008100e800e1bf9f0027
:1054700010199000efb89700810f5100d7ff3e0040
:0c5480005fb897000080fa0000000600f2
:020000040000fa
:10548c0000818200e20f5000010032000000060093
:10549c00f08082000048a300fcff3a00f0808200fc
:1054ac000018a300f9ff32008030ec00008480006b
:1054bc00e70f50002000360010848000918282009b
:1054cc00008040001084880030848000a18282001b
:1054dc000080400030848800108480004300de008f
:1054ec0010848800308480004300de003084880003
:1054fc008089820011848000004990000148980046
:10550c00c808de001049900011489800208a8200db
:10551c00318480000049900001489800c808de00e2
:10552c001049900011489800f08082000040a000c3
:10553c00f0808a00000006001084800091828200b6
:10554c00008040001084880030848000a18282009a
:0c555c0000804000308488000000060041
:020000040000fa
:105568000200fa0010002000f0bf9f00062eef0096
:1055780080002000107188003e2eef001070880017
:1055880051392000f170880071002000d171880025
:105598000070880050382000e0708800c1718800d1
:1055a8003e8ea9003a8ea9003eaea9003aaea900e7
:1055b800234ea9001f4ea9000000eb005105200052
:1055c800b1468800a10a2000b1468800006888001a
:1055d80000fc2f00860db6002002b300306c880056
:1055e800f00f2c00216c80000101600001302200c6
:1055f80082807000216c8800820db6000080a000b7
:10560800106c880040c2b30028edb700008020006d
:1056180051052000b1468800a10a2000b146880043
:10562800006888007fb897000080fa000000060034
:020000040000fa
:105638000200fa0010002000f0bf9f00e0012500e2
:10564800ccfa0700ffb8970001006000f0bf9f0088
:10565800e001250085f20700ffb89700010060000f
:10566800f0bf9f00b8fd0700ffb897000100600079
:10567800f0bf9f002007250047f60700ffb89700f6
:1056880001006000f0bf9f00e005250042f607001a
:10569800ffb8970001006000f0bf9f006008250078
:1056a8003df60700ffb8970001006000f0bf9f00bb
:1056b800a009250038f60700ffb897000100600030
:1056c800f0bf9f00e00a250033f60700ffb89700f7
:1056d80001006000f0bf9f00e00125000101070004
:1056e800ffb8970001006000f0bf9f007fb89700e7
:0856f8000080fa00000006002a
:020000040000fa
:105700000200fa0012002000f2bf9f0090029000f9
:1057100003e02000c4e120000302520085a2b9008a
:1057200083004200b00190000300e000110032004d
:10573000614290000482fb00f1419000c819dd0035
:1057400083017200200090000011dd000281ea0058
:105750000301610061409000e24098004811de00c2
:1057600071409000f24098007fb897000080fa00e6
:1057700000000600614290000482fb00f1419000ad
:10578000c819dd0083017200200090000011dd00c7
:105790000281710061409000e24098004811de00f3
:1057a00071409000f24098007fb897000080fa00a6
:0857b00000000600efff3700c6
:020000040000fa
:1057b8000200fa0012002000f2bf9f009002900041
:1057c80003e02000c4e120000302520085a2b900d2
:1057d80083004200b00190000300e0001000320096
:1057e800614290000482fb00f1419000c819dd007d
:1057f80083017200200090000011dd000281710019
:1058080061409000e24098004811de00714090002d
:10581800f24098007fb897000080fa000000060068
:10582800614290000482fb00f1419000c819dd003c
:1058380083017200200090000011dd000281ea005f
:105848000301610061409000e24098004811de00c9
:1058580071409000f24098007fb897000080fa00ed
:0858680000000600eeff37000e
:020000040000fa
:105870000200fa0010002000f0bf9f0072f3070042
:10588000ffb8970001006000f0bf9f0006ef07001f
:10589000ffb8970001006000f0bf9f0066ff07009f
:1058a000ffb8970001006000f0bf9f00e0012500f5
:1058b000f6fb0700ffb8970001006000f0bf9f00f3
:1058c0007fb897000000e00003003200f080820003
:1058d0000020a000f0808a0010000700ffb89700a9
:1058e00001006000f0bf9f00f02ba80080ff2f0098
:1058f0006e08b6005000b300704388000b88a90002
:105900002b88a800f080820000f0a000f0808a00c0
:0c5910007fb897000080fa00000006003d
:020000040000fa
:10591c000600fa0010002000d0bf9f000000eb0032
:10592c00e0bf9f00f0bf9f0001eba8008a10f800b9
:10593c00000cf900508480004800dd008a10b7008c
:10594c00f0bf9f00036080007fb997006fb897008d
:10595c008000e800e1bf9f0071382100810f5000ea
:10596c000a0036006fb997000000eb007138210077
:10597c00810f510003003e008a10f8000a0bf90059
:10598c005fb897000080fa0000000600828f51007b
:10599c00f4ff3200036080007fb997006fb8970066
:1059ac008000e800e1bf9f0071382100810f50009a
:0859bc00ecff3e00f5ff37008f
:020000040000fa
:1059c4000200fa000000eb00f0bf9f008fefa90077
:1059d400f0cf2f00922fb60000fc2f008e0fb600e0
:1059e4000000a000707c8800d1072000b0210a00cc
:1059f400900f0000f0f82f00920fb6000050a000a6
:105a0400907c880080ff2f00920fb6000000a00059
:105a1400907c88008f0fa8008fefa8000000eb0097
:105a24008e0fe20009003d008fcfab0006003a0064
:105a34007fb897008000e800f1bf9f007138210013
:105a4400810f5000f8ff3600100020000080fa009b
:045a54000000060048
:020000040000fa
:105a58000200fa0011c0b300e1ff9f00900190001e
:105a680001e02000c2e12000010151008391b9004a
:105a780001014100c24190008381fb005241900026
:105a88004811dd0002817100a00090001300200081
:105a98008118dd008280600001f0a7008100ea0023
:105aa8008100ea00cf08de00e1ff9f00300090008f
:105ab800830f5000030032006ff897000080fa004f
:105ac80000000600eff897000180fb0000805100fd
:105ad800e0ff9f006ff897000080fa0000000600c2
:045ae800f8ff37008c
:020000040000fa
:105aec000200fa00881f78000004780010002000e3
:105afc00e0bf9f0008e091000004e00010003a00b5
:105b0c0028e891000004e00004003a006fb8970008
:105b1c004f0478000080fa0000000600a00e200060
:105b2c0008004000bffb0700e0bf9f006fb8970064
:105b3c004f0478000080fa0000000600f7ff3700e1
:105b4c00000e200008004000b6fb0700e0bf9f00dd
:105b5c0028e891000004e000ecff3200efff370072
:020000040000fa
:105b6c000200fa0010002000f0bf9f00e014250096
:105b7c0080f60700ffb8970001006000f0bf9f009f
:105b8c00401625007bf60700ffb897000100600067
:105b9c00f0bf9f00a017250076f60700ffb897000e
:105bac0001006000f0bf9f000019250071f607008e
:105bbc00ffb8970001006000f0bf9f00601a25003d
:105bcc006cf60700ffb8970001006000f0bf9f0063
:0c5bdc007fb897000080fa00000006006f
:020000040000fa
:105be8000200fa0010002000f0bf9f00000820000b
:105bf800c01188003a22ef003c22ef002002270063
:105c0800f0118800b0a22000001288004222ef00a4
:105c18004c22ef004e22ef005022ef005222ef00fc
:105c28005422ef005622ef005822ef005a22ef00cc
:105c38005c22ef0039e2a80038a2a8003882a80048
:0c5c48007fb897000080fa000000060002
:020000040000fa
:105c540001e1a90001a1a9000181a9000161a90034
:105c64000141a900003020000021b70000e1a90093
:105c7400f0fc2f000021b6000041a9000021a9007a
:105c84000421ef00f070220040088800f0f82f0093
:105c94004028b6000028a9002028a900100005000b
:020000040000fa
:105ca4000200fa008000eb00f1bf9f004059900011
:105cb400d0599000e05890008381fb000281fb00e2
:105cc400028141008180fb0081004100f1bf9f00ff
:105cd400ffb8970001609800100020000080fa00cf
:045ce40000000600b6
:020000040000fa
:105ce8000200fa00881f780018002000e8bf9f0013
:105cf800e00125001cfd0700efb8970001006000d7
:105d0800e0bf9f00e00125001070a00008818a0014
:105d18006fb897004f0478000080fa000000060072
:020000040000fa
:105d2800a005250020988a000080e90030988a00a4
:105d38006600500040988a000080e80050988a0069
:105d4800403225000008eb004002b1001010a1000d
:0c5d58001030a10010f0a00010000500a9
:020000040000fa
:105d64000200fa0010002000f0bf9f000030250060
:105d740087f30700ffb8970001006000f0bf9f00a1
:0c5d84007fb897000080fa0000000600c5
:020000040000fa
:105d900050998a00c03225001008e8000000000079
:105da00000000000000000000000000000000000f3
:085db0000000000000000600e5
:020000040000fa
:105db8000200fa000000eb00f0bf9f001000200076
:105dc80000818a00e001250010f0a0007fb897004c
:085dd8000080fa000000060043
:020000040000fa
:020000040005f5
:047e0000ffffff0081
:020000040000fa
:020000040005f5
:047e2000ffffff0061
:020000040000fa
:020000040005f5
:047e3000f8ffff0058
:020000040000fa
:020000040005f5
:047e38007bffff00cd
:020000040000fa
:020000040005f5
:047e4000ff7fff00c1
:020000040000fa
:020000040005f5
:047e4800ffffff0039
:020000040000fa
:020000040005f5
:047e5000deffff0052
:020000040000fa
:020000040005f5
:047e5800ffffff0029
:020000040000fa
:020000040005f5
:047e6000ffffff0021
:020000040000fa
:020000040005f5
:047e6800ffffff0019
:020000040000fa
:020000040005f5
:047e7000ffffff0011
:020000040000fa
:020000040005f5
:047e7800ffffff0009
:020000040000fa
:020000040005f5
:047e8000fffcff0004
:020000040000fa
:020000040005f5
:047e8800fcffff00fc
:020000040000fa
:020000040005f5
:047ff800ffffff0088
:00000001FF
